:100000003928A000A00DA00D200D3839C1389F005F
:100010000030A100323020201F151F190D28A1012A
:100020001E083428A301A200FF30A207031CA30767
:10003000031C34280330A100DF3020201428A10144
:10004000E83EA000A109FC30031C2928A0070318E2
:100050002628A0076400A10F262820182F28A01CFE
:10006000332800003328080083130313831264002D
:100070000800FF2383168F00831283161F3085002C
:1000800002309F008312BB010A3012206400051A5F
:100090004E28851283168512831244280A301220B6
:1000A00000300120BF0001303F07B200B301B30DA3
:1000B00005303207BF000A30122001300120BD0098
:1000C0000230BD070A30122002300120BE00640059
:1000D0003B08013C031D702805303F02C000722818
:1000E0003F08C000640040083E0203187D28BB01A1
:1000F000851283168512831244280130BB006400E8
:10010000851987288512831685128312442885163F
:100110008316851283120130BC0064003C083D0246
:10012000031C9B280730A300D03013206400051E59
:0C0130004428BC0F8D28442863009C2844
:02400E006C3F05
:00000001FF
